:100000000C9411050C9449050C9449050C94490570
:100010000C9449050C9449050C9449050C94490528
:100020000C9449050C9449050C9449050C943B2605
:100030000C94EA260C94AC200C9449050C944905C8
:100040000C9449050C9449050C9449050C943421F1
:100050000C9449050C9449050C9449050C944905E8
:100060000C9449050C9449050C9449050C944905D8
:100070000C94490504090409300930099809B609A6
:10008000CE0ACE0AC1095A0A6B0A6B0A57277E2785
:1000900076287E277628CA27ED27762844285328F5
:1000A000165C1F0021002300250027002E002A00D7
:1000B0001E0020002200240026002D0031004900EF
:1000C0002B001A0015001C000C001300300000006B
:1000D000140008001700180012002F0031004C0017
:1000E000E400160009000B000E00330000000000C1
:1000F000040007000A000D000F00340028004B0028
:10010000E1001B0019001100360038000000520009
:100110001D0006000500100037000000E5004E003D
:10012000E000E200000000000000E600E4005100F2
:10013000E30000002C0000000000E70050004F002A
:1001400044454255473A2064697361626C65642E88
:100150000A0044454255473A20656E61626C656409
:100160002E0A000A0025303258006C65645F746105
:10017000736B3A20004F6E6573686F743A20616349
:10018000746976653A2025640A000A0025303862D1
:10019000003A200025303258000A722F6320303197
:1001A0003233343536370A00290A002575002F000E
:1001B0002575005D280025640020002564002000CE
:1001C00025640020002564007C0025303258006D35
:1001D0006F7573656B6579205B62746E7C782079CE
:1001E000207620685D287265702F61636C293A2043
:1001F0005B00313A0964656C6179282A31306D738E
:10020000293A2025750A323A09696E746572766159
:100210006C286D73293A2025750A333A096D617887
:100220005F73706565643A2025750A343A0974690C
:100230006D655F746F5F6D61783A2025750A353A98
:1002400009776865656C5F6D61785F73706565647B
:100250003A2025750A363A09776865656C5F7469D6
:100260006D655F746F5F6D61783A2025750A007067
:100270003A097072696E742076616C7565730A64F0
:100280003A097365742064656661756C74730A75E8
:10029000703A092B310A646E3A092D310A6C743AAE
:1002A000092B31300A72743A092D31300A45534313
:1002B0002F713A09717569740A0A73706565642053
:1002C0003D2064656C7461202A206D61785F7370D5
:1002D000656564202A2028726570656174202F206E
:1002E00074696D655F746F5F6D6178290A77686501
:1002F00072652064656C74613A20637572736F7205
:100300003D25642C20776865656C3D25640A53653E
:100310006520687474703A2F2F656E2E77696B694B
:1003200070656469612E6F72672F77696B692F4DF5
:100330006F7573655F6B6579730A004D3E20004DE4
:1003400025753A25733E20003F0A003D2025750A99
:10035000003F0A0064656661756C74730A00257558
:100360000A003F0A000A092D2056616C756573204A
:100370002D0A00710A000A092D204D6F7573656BF7
:100380006579202D0A003F00433E20004C25640A79
:10039000000A092D20537461747573202D0A686F4B
:1003A00073745F6B6579626F6172645F6C656473AF
:1003B00028293A20253032580A6B6579626F6172BC
:1003C000645F70726F746F636F6C3A2025303258BF
:1003D0000A6B6579626F6172645F69646C653A206B
:1003E000253032580A74696D65725F7265616433D5
:1003F0003228293A202530386C580A000A092D2065
:1004000056657273696F6E202D0A5649443A203042
:100410007846454544285377697463686D6F642056
:100420004B6579626F6172647329205049443A20A8
:10043000307830303030284D656D65292056455272
:100440003A203078303030310A4255494C443A2015
:1004500020284665622032382032303232290A4F55
:100460005054494F4E533A204C554641204D4F551C
:1004700053454B45592045585452414B455920430B
:100480004F4E534F4C4520434F4D4D414E44203429
:100490003039360A4743433A20352E342E30204136
:1004A00056522D4C4942433A20322E302E302041B4
:1004B00056525F415243483A2061767233350A0002
:1004C0000A092D20436F6E736F6C65202D0A45530A
:1004D000432F713A09717569740A6D3A096D6F7528
:1004E00073656B65790A000A092D204D61676963A0
:1004F000202D0A443A094465627567204D6573737F
:1005000061676520546F67676C650A583A094D61E9
:1005100074726978204465627567204D6F64652048
:10052000546F67676C65202D2053686F77206B656B
:10053000797072657373657320696E206D61747272
:10054000697820677269640A4B3A094B6579626F72
:1005500061726420446562756720546F67676C65DB
:10056000202D2053686F77206B65797072657373E7
:10057000207265706F72740A4D3A0944656275673E
:10058000204D6F75736520546F67676C650A563A26
:100590000956657273696F6E0A533A095374617430
:1005A00075730A433A09416374697661746520433F
:1005B0006F6E736F6C65204D6F64650A46312D4612
:1005C00031303A0953776974636820746F204C6145
:1005D00079657220302D392028463130203D204C5D
:1005E00030290A302D393A095377697463682074C9
:1005F0006F204C6179657220302D390A475241567F
:10060000453A0953776974636820746F204C6179A7
:10061000657220302028616C7465726E6174652982
:100620000A423A094A756D7020746F20426F6F74E8
:100630006C6F616465720A4553433A094A756D707F
:1006400020746F20426F6F746C6F61646572202834
:10065000616C7465726E617465290A453A0950725D
:10066000696E7420454550524F4D2053657474692E
:100670006E67730A4253504143453A09436C6561C2
:100680007220454550524F4D0A006B65796D61707F
:100690005F636F6E6669672E7261773A202530322C
:1006A000580A2E737761705F636F6E74726F6C5F40
:1006B000636170736C6F636B3A2025750A2E6361FA
:1006C00070736C6F636B5F746F5F636F6E74726F68
:1006D0006C3A2025750A2E737761705F6C63746CB9
:1006E0005F6C6775693A2025750A2E737761705FB4
:1006F0007263746C5F726775693A2025750A2E7390
:100700007761705F6C616C745F6C6775693A202506
:10071000750A2E737761705F72616C745F726775B2
:10072000693A2025750A2E6E6F5F6775693A202534
:10073000750A2E737761705F67726176655F6573A6
:10074000633A2025750A2E737761705F6261636B6F
:10075000736C6173685F6261636B73706163653A48
:100760002025750A2E6E6B726F3A2025750A00647B
:10077000656275675F636F6E6669672E7261773A4F
:1007800020253032580A2E656E61626C653A20254C
:10079000750A2E6D61747269783A2025750A2E6B80
:1007A0006579626F6172643A2025750A2E6D6F75E6
:1007B00073653A2025750A006565636F6E66696723
:1007C0003A0A64656661756C745F6C617965723A4A
:1007D0002025750A003F000A6D6F7573653A206F1A
:1007E00066660A000A6D6F7573653A206F6E0A00BF
:1007F0000A6B6579626F6172643A206F66660A00FF
:100800000A6B6579626F6172643A206F6E0A000A42
:100810006D61747269783A206F66660A000A6D61CC
:10082000747269783A206F6E0A000A6465627567AF
:100830003A206F66660A000A64656275673A206F3F
:100840006E0A000A0A4A756D70696E6720746F201F
:10085000626F6F746C6F616465722E2E2E20004380
:100860003E2000436C656172696E672045455052B9
:100870004F4D0A000A002530325820006B6579621E
:100880006F6172645F7265706F72743A20005B739F
:100890005D005B575D005B535D005B525D000A03CA
:1008A0004D0065006D0065000000280353007700CF
:1008B00069007400630068006D006F006400200030
:1008C0004B006500790062006F00610072006400F7
:1008D000730000000403090409025B00030100A087
:1008E000FA090400000103010100092111010001BE
:1008F00022400007058103080001090401000103EB
:10090000000000092111010001227B00070582037C
:100910002000010904020002030000000921110166
:1009200000012222000705830320000107050303BD
:100930002000011201000200000008EDFE0000018D
:1009400000010200010631FF0974A10109751500BB
:1009500026FF009520750881020976150026FF0004
:10096000952075089102C005010902A101850209BF
:1009700001A100050919012908150025019508752F
:100980000181020501093009311581257F95027524
:1009900008810609381581257F95017508810605AE
:1009A0000C0A38021581257F950175088106C0C0A3
:1009B00005010980A101850319012AB70015012647
:1009C000B700950175108100C0050C0901A10185D2
:1009D0000419012AA002150126A0029501751081B3
:1009E00000C005010906A101050719E029E7150066
:1009F000250195087501810295017508810105079A
:100A0000190029FF150026FF0095067508810005CD
:100A10000819012905950575019102950175039144
:100A200001C011241FBECFEFD4E0DEBFCDBF04B69E
:100A300003FE18C08091F0029091F102A091F202A1
:100A4000B091F3028730904BA740B04B59F410920D
:100A5000F0021092F1021092F2021092F302E0E022
:100A6000F8E3099511E0A0E0B1E0ECE9F2E502C09D
:100A700005900D92AA3FB107D9F722E0AAEFB1E0A5
:100A800001C01D92A03FB207E1F70E94EE160C9440
:100A90004C290C940000FF93EF93E091FA01F09140
:100AA000FB01309709F00995EF91FF910895FC0142
:100AB0008591803011F0EFDFFBCF0895FF27E0E252
:100AC00030E247FF0CC0419597FF09C0EDE2609509
:100AD000709580959095611D711D811D911D27FF59
:100AE00002C0219530E350E2AA27660F771F881FC6
:100AF000991FAA1FA41710F0A41B63955A95A9F774
:100B0000AA3008F0A95FA05DAF93F3956115710558
:100B10008105910541F7ED3211F4EF93F395F2174A
:100B200018F43F93F395FBCF8F91B5DFFA95E1F77A
:100B30000895E991F9918591803021F0853219F07D
:100B4000AADFF9CF089520E0E89455915532C1F31A
:100B5000503311F4689455915A3348F4505390F33C
:100B6000220F022E220F220F200D250FF4CF0EF49C
:100B7000219589919991533619F3533729F15335BA
:100B800059F1BC0188279927E8945C3621F48991B2
:100B9000999168945591543639F446EF7EF077FF79
:100BA0000DC08FEF9FEF0AC055374AE039F0583536
:100BB00040E121F0523642E009F00895FF93EF93AF
:100BC0007DDFEF91FF91B7CFFF93EF93FC01819110
:100BD0008030B9F360DFFBCFFF93EF9368DFF1CF95
:100BE000DF93CF93CDB7DEB72596A3DFCF91DF910B
:100BF000089581E0089581E008950C94FB0508951F
:100C00000C94FF051F93CF93DF9300D000D01F9269
:100C1000CDB7DEB749835A836B833091FD0189815B
:100C20009A81311114C0662359F0222349F00E94A1
:100C3000100D182F682F89819A810E94B40C03C06F
:100C40000E94E30C182F69817A81812F04C00E94D1
:100C5000100D69817A810F900F900F900F900F9077
:100C6000DF91CF911F910C943B14FC01262F408102
:100C700051816281738184810C94020681E0089520
:100C8000CF93DF93EC0160E00E943506BE01DF9157
:100C9000CF910C9400060C94AE150C94AA150895EF
:100CA0000E945E0B0E944F062FEF84E39CE02150D0
:100CB00080409040E1F700C000000C945A210F934F
:100CC0001F93CF93DF938C0161E00E943506EC0106
:100CD000B8010E94FD05882309F45BC0B801CE016C
:100CE0000E943A1F882309F454C0B801CE010E9423
:100CF0001C1A882309F44DC0B801CE010E94961E2B
:100D0000882309F446C0F80182818823D9F1CF3DB8
:100D10008CE5D80779F140F4C115FCE5DF0791F0C7
:100D2000C130DC4591F02EC0CC35EDE5DE0741F158
:100D3000CD35FDE5DF0709F1CB35DD4519F50E941D
:100D4000A31120C00E94500624C080919602C82F93
:100D5000C095C170C0FB80F980939602CC2329F026
:100D600082E591E00E94570514C080E491E00E9462
:100D7000570510C00E9451120CC00E949A1102C067
:100D80000E94A611C801DF91CF911F910F910C9481
:100D9000F905C0E08C2FDF91CF911F910F9108953D
:100DA0000E948F200C94FB060E94FE060C94952056
:100DB0008295982F9373292F220F220F982F9C7CB6
:100DC00096959695922B892F8575880F9A7A969588
:100DD000892B089508950C94EA0681E008950C94F7
:100DE000ED060895CF93C82F0E94EB068C2F0E942A
:100DF000EF06CF91089580E00C94F2060E94961FB2
:100E00000C94F206CF930E94961FC82F8091FC018C
:100E1000C81741F1C093FC018091960282FF1EC069
:100E200080FF04C08AE691E00E94570580919602F7
:100E300080FF0CC01F92CF9385E691E09F938F9324
:100E40000E94F0050F900F900F900F9080919602E6
:100E500080FF04C083E691E00E9457058C2FCF915C
:100E60000C94F206CF910895CF93DF93CDB7DEB700
:100E70002B970FB6F894DEBF0FBECDBF4F835887B8
:100E800069877A878B8761110E94D2109E012F5F3C
:100E90003F4F86E0F90111928A95E9F785E0FE015E
:100EA0003796D90101900D928A95E1F789819A814F
:100EB0004C815D81452B31F09F3F31F491E08F3FB4
:100EC00019F403C091E001C090E090FF09C049818E
:100ED0005A816B817C818D819E810E94EE0F05C0BD
:100EE000C9010E943E068111F2CF2B960FB6F894ED
:100EF000DEBF0FBECDBFDF91CF910895FC01808191
:100F000091810E94520D0895CF93882309F4A9C0BE
:100F1000C82F8238C1F40E94961F81FDA2C069E3E8
:100F200080910201909103010E9467200E94F410B9
:100F30002FEF81EE94E0215080409040E1F700C017
:100F4000000069E319C0833801F50E94961F80FDF7
:100F500088C063E580910201909103010E9467209F
:100F60000E94F4102FEF81EE94E0215080409040D9
:100F7000E1F700C0000063E5809102019091030158
:100F80000E946920CF910C94F4108438C1F40E941F
:100F9000961F82FD66C067E4809102019091030173
:100FA0000E9467200E94F4102FEF81EE94E0215000
:100FB00080409040E1F700C0000067E4DDCF8CEF97
:100FC0008C0F813AF8F48C2F0E943F1E811149C08A
:100FD0006C2F80910201909103010E94312088239F
:100FE00049F06C2F80910201909103010E946920C9
:100FF0000E94F4106C2F80910201909103010E94D5
:101000006720C0CF80E28C0F883048F4C77081E041
:1010100001C0880FCA95EAF70E94B510B3CFEBE57F
:10102000EC0FE33040F4F0E0E95BFE4F808190E0AC
:10103000CF910C94F91FE8E5EC0FE73150F4F0E0A4
:10104000EE0FFF1FE75EFE4F80819181CF910C94E0
:101050000F20CD3E30F08C2F0E947B17CF910C9447
:101060004D18CF910895882309F464C0823879F42B
:101070000E94961F81FF5EC069E3809102019091FA
:1010800003010E9467200E94F41069E310C08338B6
:10109000B1F40E94961F80FF4DC063E5809102016C
:1010A000909103010E9467200E94F41063E58091F3
:1010B0000201909103010E9469200C94F41084387D
:1010C00079F40E94961F82FF35C067E48091020187
:1010D000909103010E9467200E94F41067E4E7CF1B
:1010E0009CEF980F913A10F4682FE1CF90E2980F9F
:1010F000983050F4877091E001C0990F8A95EAF713
:10110000892F0E94BB10D9CF9BE5980F933020F414
:1011100080E090E00C94F91F98E5980F973120F447
:1011200080E090E00C940F208D3E20F00E94D617B6
:101130000C944D1808951F93CF93DF93182FEB0154
:101140000E948407209741F08FE99FE00197F1F713
:1011500000C000002197F6CF812FDF91CF911F9122
:101160000C943308893319F060E070E002C060E548
:1011700070E00C949B08882321F00E94B5100C9419
:10118000F4100895882321F00E94BB100C94F410F1
:101190000895CF92DF92EF92FF920F931F93CF9318
:1011A000DF937C01D62FC72FFC01128105810295A8
:1011B0000F700E94AB108823B9F01123A9F08C2F77
:1011C000807F803421F080E28D0F883068F080913C
:1011D000CA0282FD09C082E00E9454110E94AB1035
:1011E00091E0D82ED92601C0D12CCC2EC2948FE00C
:1011F000C8228C2D90E08C30910508F0CFC1FC0105
:10120000E65CFF4F0C94E3288C2F807FCF708823FF
:1012100011F0C295C07F112399F0CC2309F4AAC123
:1012200080E28D0F883010F0D11104C08C2F0E9405
:10123000B51003C08C2F0E94C5100E94F4109AC1F3
:101240008D2F0E943308CC2309F4A8C180E28D0FB2
:10125000883038F1DD2329F18C2F0E94CB1024C077
:101260008C2F807FCF70803211F0C295C07FDD233C
:1012700019F0D130A1F13DC08091CA0282FF17C0A0
:10128000112349F0CC2329F08C2F0E94B5100E9425
:10129000F41080E070C180E00E943308CC2309F490
:1012A0007DC18C2F0E94BB100E94F41077C11123C6
:1012B00071F0002341F0013031F40E94D5108C2BE5
:1012C0000E94DD106BC10E94D5108C2B1DC0002325
:1012D00019F0013009F462C10E94EA1025C01123FF
:1012E00021F0063008F05AC10EC0053008F056C192
:1012F0001BC0112361F0002331F0F701858180FFCD
:1013000039C18F7085838C2F0E94BB0847C1002391
:1013100059F0D93309F03FC1FFEF07EE13E0F15068
:1013200000401040E1F735C18C2F0E94C20836C141
:101330008C2F86958695837019F0813061F02EC1CF
:10134000112321F08D2F9C2F937002C080E090E03C
:101350000E94F91F2BC1112321F08D2F9C2F937018
:1013600002C080E090E00E940F2020C18D2F112349
:1013700019F00E947B1702C00E94D6170E944D18D8
:1013800015C18C2F837009F047C011110BC12D2F8F
:10139000229526952770220F220F6D2F6F70862FB2
:1013A00090E0A0E0B0E0022E04C0880F991FAA1FB1
:1013B000BB1F0A94D2F7D4FF10C04FE050E060E0AA
:1013C00070E004C0440F551F661F771F2A95D2F79F
:1013D000409550956095709503C040E050E0BA018B
:1013E000C695C695C3708A019B01082B192B2A2B21
:1013F0003B2BC901B801C23049F058F4C13019F093
:101400000E94CA0BCFC00E94B80BCCC00E94DC0B5C
:10141000C9C00E94B60BC6C0112319F08C2F817071
:1014200001C08695882309F4BDC02D2F22952695ED
:101430002770220F220F6D2F6F70862F90E0A0E093
:10144000B0E0022E04C0880F991FAA1FBB1F0A9488
:10145000D2F7D4FF10C04FE050E060E070E004C06D
:10146000440F551F661F771F2A95D2F74095509558
:101470006095709503C040E050E0BA01C695C695EE
:10148000C3708A019B01082B192B2A2B3B2BC90106
:10149000B801C23049F058F4C13019F00E948F0CE5
:1014A00081C00E947D0C7EC00E94A10C7BC00E9466
:1014B000F00B78C0CF70112339F08C2F0E94160CDE
:1014C0008D2F0E94BB086EC08D2F0E94C2088C2FEA
:1014D0000E94370C67C0D23F21F128F4D03F41F081
:1014E000D13FC1F043C0D33F19F1D43F79F03EC0A2
:1014F000112341F0053008F051C08C2F8F710E94EC
:101500005C0C4CC0063008F049C0F7CF8091CA028D
:1015100082FF18C0112339F08C2F8F710E94160C96
:101520003DC01123C9F38C2F8F710E94370C36C038
:10153000112329F08C2F8F710E94010C2FC00E9463
:10154000FC0B2CC0112349F0CF718C2F0E94160C7C
:1015500063E08C2F0E94391121C081E00E94541158
:101560000230E0F082E00E94541118C0112331F0E3
:10157000002391F28D2F0E94840710C0002399F25E
:10158000D93349F41FEF27EE33E0115020403040AB
:10159000E1F700C000008D2F0E94330888EF8C0D0A
:1015A000843020F40E94961F0E94F206DD20C9F0CC
:1015B0000E94A71080FD15C0F70112820E94A110A1
:1015C0000E94160CC7010E94120B0E94A110DF910D
:1015D000CF911F910F91FF90EF90DF90CF900C94DF
:1015E000370CDF91CF911F910F91FF90EF90DF901B
:1015F000CF9008950F931F93CF93DF93EC016881F1
:1016000079818A810E945D0D8C010E94B30C0E9439
:10161000A40BB801CE010E94C908DF91CF911F91A0
:101620000F910895CF93DF93EC01988189812B81ED
:101630003C81232B31F08F3F31F481E09F3F19F43F
:1016400003C081E001C080E080FD1DC0CE010E948A
:101650005F06811110C00E94AB108823A1F08A811F
:10166000882389F08091CA0282FD0DC082E0DF915B
:10167000CF910C945411CE010E94FA0ACE01DF9151
:10168000CF910C944006DF91CF91089580E090E0D7
:101690000E94F91F80E090E00E940F200E94D2106B
:1016A0000E94F4100E940E1A0C944D1880910201B1
:1016B000909103010E946B200C94460B0E94C21073
:1016C0000C94560B92959F70963079F010F49250CE
:1016D00001C09A50923068F4803F69F018F4883E57
:1016E00040F409C0843F29F406C0883E20F0813FC1
:1016F00011F080E0089581E00895FC0180819181DE
:101700000E94520D0E94620B0895CF93DF9300D088
:1017100000D01F92CDB7DEB70F900F900F900F90B3
:101720000F90DF91CF910895CF93DF9300D000D039
:1017300000D0CDB7DEB726960FB6F894DEBF0FBE49
:10174000CDBFDF91CF910895089508950C94A50B16
:101750000C94A60B0E94A80B609334027093350280
:1017600080933602909337020C94460B0C94AA0B8C
:101770000F931F930091340210913502209136028D
:1017800030913702602B712B822B932B1F910F917D
:101790000C94AA0B0F931F93009134021091350201
:1017A00020913602309137026023712382239323E4
:1017B0001F910F910C94AA0B0F931F930091340269
:1017C000109135022091360230913702602771273F
:1017D000822793271F910F910C94AA0B0C94A50BB1
:1017E0000E94EE0B609330027093310280933202BC
:1017F000909333020C94460B60E070E0CB010C94A4
:10180000F00B0F931F9341E050E060E070E08A011D
:101810009B0104C0000F111F221F331F8A95D2F7AE
:10182000C901B8011F910F910C94F00B0F931F93F6
:1018300041E050E060E070E004C0440F551F661FB7
:10184000771F8A95D2F78091300290913102A09152
:101850003202B09133028A019B01082B192B2A2BEB
:101860003B2BC901B8011F910F910C94F00B0F9302
:101870001F9341E050E060E070E004C0440F551F4A
:10188000661F771F8A95D2F74095509560957095A1
:101890008091300290913102A0913202B0913302D6
:1018A0008A019B01082319232A233B23C901B8017C
:1018B0001F910F910C94F00B0F931F9341E050E098
:1018C00060E070E004C0440F551F661F771F8A95C3
:1018D000D2F78091300290913102A0913202B09102
:1018E00033028A019B01082719272A273B27C901B0
:1018F000B8011F910F910C94F00B0F931F9300915F
:101900003002109131022091320230913302602B6B
:10191000712B822B932B1F910F910C94F00B0F9333
:101920001F930091300210913102209132023091C8
:10193000330260237123822393231F910F910C9410
:10194000F00B0F931F930091300210913102209100
:1019500032023091330260277127822793271F912B
:101960000F910C94F00B0895262F990F990F990F52
:10197000890F982F9770A1E001C0AA0F9A95EAF7F6
:1019800086958695869590E065E070E00E94B22885
:10199000FC01E250FE4F40E050E0622F70E0908189
:1019A0009B01042E02C0369527950A94E2F7217018
:1019B000219529272A23292721934F5F5F4F4530FF
:1019C000510569F70895990F990F990F890FA82F5D
:1019D000A77086958695869590E065E070E00E94F8
:1019E000B228BC0140E050E080E0FB01E40FF51FAD
:1019F000E250FE4F208130E00A2E02C03695279536
:101A00000A94E2F721703327042E01C0220F0A94B2
:101A1000EAF7822B4F5F5F4F4530510531F708954C
:101A2000BF92CF92DF92EF92FF920F931F93CF93CB
:101A3000DF938C01C0903002D0903102E0903202EE
:101A4000F09033028091340290913502A0913602D9
:101A5000B0913702C82AD92AEA2AFB2ACFE1D0E07E
:101A6000D701C6010C2E04C0B695A795979587950A
:101A70000A94D2F780FD04C0219790F7B12C07C0DB
:101A8000BC2EB8018C2F0E9452140197A9F38B2D04
:101A9000DF91CF911F910F91FF90EF90DF90CF904A
:101AA000BF900895CF93DF93EC010E94100DBE010B
:101AB0000E945214DF91CF9108951F93CF93DF932B
:101AC000EB019091FD01992321F0CB010E94520D71
:101AD00013C0882349F0CB010E94100D182F682FE6
:101AE000CE010E94B40C04C0CB010E94E30C182F5D
:101AF000BE01812F0E945214DF91CF911F91089552
:101B0000CF93DF93C091380280913902C817A1F0BA
:101B1000D0E0CE0166E070E00E94B228FC01E65CF5
:101B2000FD4F4081518162817381848195810E9442
:101B3000940B2196C770E8CFDF91CF910895409123
:101B40006A0250916B0260916C0270916D028091FB
:101B50006E0290916F020C94940BFF920F931F935F
:101B6000CF93DF9380916F0282958F7009F062C0EE
:101B700080916C02882309F45DC020913802F090B6
:101B8000390210916A0200916B02A0916D02B0912E
:101B90006E0281E01F3F09F080E0C0910001D0910A
:101BA0000101482F2F1509F445C0109721F00F3F70
:101BB00021F080E003C081E001C0842F30E080FD8F
:101BC00035C0C90166E070E00E94B228FC01E65C05
:101BD000FD4F818180132AC08081811327C08281BB
:101BE000811124C0838194818A1B9B0B8C179D07D4
:101BF000E8F480916F028F70806180936F02C90159
:101C000066E070E00E94B228FC01E15CFD4F90812B
:101C10009F70906190838AE692E00E94120BDF91A0
:101C2000CF911F910F91FF900C94800D2F5F3F4F2C
:101C30002770B8CFDF91CF911F910F91FF9008953A
:101C40009F92AF92BF92CF92DF92EF92FF920F934B
:101C50001F93CF93DF93CDB7DEB761970FB6F8949C
:101C6000DEBF0FBECDBF8C0185E0F801DE011D9601
:101C700001900D928A95E1F7F801E28090916A0255
:101C800030916B0260916D0270916E026115710569
:101C900031F03F3F31F481E09F3F19F403C081E010
:101CA00001C080E0F82FF1709F2E80FD47C1F80140
:101CB00040812181A380B4808AE6C82E82E0D82E9C
:101CC000F0906C02F501E61BF70B6091000170913A
:101CD0000101FF2009F4DCC080916F02582F507F72
:101CE000E617F70708F096C0511155C0231313C02B
:101CF000491311C0FE2CE1100EC08F7080618093DB
:101D00006F020E949F0DC6010E94120B80916F020C
:101D1000F801858350C1AB2831F02F3F31F481E0C9
:101D20004F3F19F403C081E001C080E080FD03C093
:101D300081E08E2502C080E090E0F82FF170FF2E48
:101D400080FF1FC0E091380230913902E31709F497
:101D500010C1F0E0CF0166E070E00E94B228DC0123
:101D6000A65CBD4F11968C911197281307C08C91DA
:101D7000481304C012968C91E81203C03196E770A4
:101D8000E5CFFE2CEE2009F416C180916F02816030
:101D900080936F0254C0231306C0491304C0E1109E
:101DA00002C0F80199C0C8010E947D0B882361F12F
:101DB000EE2051F120916F02822F82958F7090E07A
:101DC000029774F080916A0290916B0298878F83DA
:101DD0001986BB86AA862C87CE0107960E94120B15
:101DE00086E0F801AAE6B2E001900D928A95E1F74B
:101DF0000E94AD0D0E949F0D0AC0231711F1C8016A
:101E00000E947D0B81112CC0C8010E94120BFF247F
:101E1000F394D1C05111F1CF7A2DB98AA88A522FEB
:101E20006E2D89890E94850B8AE692E00E94120B32
:101E300086E0F60111928A95E9F70E949F0DF12C38
:101E4000BAC04913DCCFE110DACFF8018583C801AD
:101E50000E94120B86E0F60111928A95E9F7ABC059
:101E6000EE2091F220916F02822F82958F7090E088
:101E700002970CF4B5CF80916A0290916B029A831D
:101E800089831B82BD82AC822E83CE010196A6CFB0
:101E9000E617F70708F044C0FE2CEE2009F4B4CF93
:101EA000231330C049132EC020916F0220FD21C0A2
:101EB000822F82958F70482F50E041155105C9F04F
:101EC000F80125834F30510541F08F5F982F92958F
:101ED000907F822F8F70892B8583C8010E94120BFF
:101EE00086E0F801AAE6B2E001900D928A95E1F74A
:101EF0003DC086E0F801AAE6B2E001900D928A9515
:101F0000E1F759C0C8010E947D0B811169CF809112
:101F10006F02816080936F02C8010E94120B4BC058
:101F20007A2DB98AA88A522F6E2D89890E94850B35
:101F300086E0F60111928A95E9F718C0EE2009F4BF
:101F400063CFC8010E947D0BF82E882309F45CCF73
:101F500086E0F801AAE6B2E001900D928A95E1F7D9
:101F60008AE692E00E947E070E94AD0D0E949F0DBE
:101F700022C04D872E878D859E850E94520D292F68
:101F800022952F70223028F49F7039F0811105C0FE
:101F90000BC0243028F49F7049F4805E883020F014
:101FA000C8010E94120B9F2CF92C05C0F8019581E5
:101FB000907F99F7F9CF8F2D61960FB6F894DEBF19
:101FC0000FBECDBFDF91CF911F910F91FF90EF908A
:101FD000DF90CF90BF90AF909F900895CF93DF9305
:101FE000CDB7DEB72C970FB6F894DEBF0FBECDBFCE
:101FF0004F83588769877A878B879C87CE0107969E
:102000000E94200E8823D1F09F8188852A853B85F8
:10201000232B31F08F3F31F481E09F3F19F403C04F
:1020200081E001C080E080FD6FC04F8158856985E7
:102030007A858B859C850E94940B66C086E0FE01A4
:102040003796DE01119601900D928A95E1F7FF8196
:10205000E8856A857B856115710531F0EF3F31F4C4
:1020600081E0FF3F19F403C081E001C080E080FD02
:102070004BC08091390290E09C012F5F3F4F277049
:1020800033274091380250E02417350709F443C044
:10209000F983EA837D836C8366E070E00E94B22856
:1020A000DC01A65CBD4F96E0FE01319601900D92D9
:1020B0009A95E1F7209339020E94800D25C090E0A7
:1020C00066E070E00E94B228865C9D4F0E94200E60
:1020D000882371F18091380290E066E070E00E9400
:1020E000B228FC01E65CFD4F408151816281738121
:1020F000848195810E94940B8091380290E0019632
:102100008770992780933802809138029091390224
:102110008913D5CF0DC00E945E0B10923902109228
:102120003802EAE6F2E086E0DF011D928A95E9F7DF
:102130002C960FB6F894DEBF0FBECDBFDF91CF91C6
:10214000089580917802859585958595089580916B
:1021500078028770089590917802977081E009F471
:1021600080E0089580918302089590918302892BE5
:1021700080938302089580959091830289238093B0
:102180008302089510928302089590918202892B10
:102190008093820208958095909182028923809392
:1021A0008202089510928202089580917902089522
:1021B00008950C94D8100C94D9109091CA0292FDF5
:1021C00008C090917902981721F0809379020C94BD
:1021D000DB10089580917902882329F0109279020A
:1021E00080E00C94DB100895CF93DF93E09102011F
:1021F000F0910301809183028083E0910201F091CC
:102200000301908180918202892B808380917902E1
:10221000882381F0E0910201F09103019081892BE4
:10222000808380910201909103010E9425208111F9
:102230000E94EA10C0910201D091030148E050E0F1
:1022400060E772E0CE010E94FD28892B69F088E0EA
:10225000FE01A0E7B2E001900D928A95E1F7CE0170
:10226000DF91CF910C94A21FDF91CF9108950C9430
:10227000D8109091CA0292FD10C0982F990F990F13
:10228000990F692B609378020E94160C8091780256
:102290008595859585950C9437110C94160C1092A4
:1022A000780280E00C943711209178028095822387
:1022B00080937802982F977099F430E0482F082E79
:1022C000000C550B2417350759F09091CA0292FD66
:1022D00007C08595859585950E94370C0C944F1104
:1022E0000895CF939091CA0292FB222720F92817D4
:1022F000F9F0C82F892FC0FB82F98093CA02809120
:10230000C9029091CA020E94CD1182E00E9454112C
:102310008091960280FF0CC01F92CF9385E791E0D9
:102320009F938F930E94F0050F900F900F900F9046
:10233000CF9108958091CA0282FB882780F991E0AD
:1023400089270C94711181E00C94711180E00C9438
:10235000711180E090E00E94122921E0893E9E4F99
:1023600009F020E0822F089582E090E00C940A2981
:1023700083E090E00C940A29CF9384E090E00E94DF
:102380000A29C82F82E290E00E940A292C2F30E00F
:10239000A901582BCA01CF910895CF93C92F682F57
:1023A00084E090E00E9418296C2F82E290E0CF91A7
:1023B0000C941829AB01BC018FE090E00C942A2901
:1023C000AB01BC0183E190E00C942A2960E070E04D
:1023D000CB010C94E01160E070E0CB010E94DA11B7
:1023E0000C94E61169EE7EEF80E090E00E943629C1
:1023F00060E082E090E00E94182960E083E090E0D5
:102400000E9418291092340210923502109236025E
:102410001092370260E084E090E00E94182960E0AA
:1024200082E290E00E94182960E085E090E00E943E
:10243000182960E086E090E00E9418296FEF87E09D
:1024400090E00E94182940E050E0BA0188E090E056
:102450000E942A2960E08DE090E00E94182940E067
:1024600050E0BA0188E190E00E942A2960E087E10B
:1024700090E00E94182940E050E0BA018CE190E021
:102480000E942A2960E070E080E290E00E943629F4
:1024900040E050E0BA0188E190E00E942A290C94C3
:1024A000EB110C94F211682F8EE090E00C94182937
:1024B0000E94192160939202709393028093940278
:1024C0009093950260938E0270938F028093900296
:1024D00090939102089581E008950C946B120895F1
:1024E0000C946F120C946F120C9472120C946F1265
:1024F0000C9476120C946F1284E393E20E948C1F6A
:102500000E947A120C9478120E9470120C946F122E
:102510000E942F150C94F1060E9404210E944B1674
:102520000E9488120C9474128F929F92AF92BF9265
:10253000CF92DF92EF92FF920F931F93CF93DF938F
:10254000CDB7DEB72A970FB6F894DEBF0FBECDBF6A
:102550000E946016982E81110E94581284E8A82EBD
:1025600082E0B82E00E010E0802E802F0E945315EC
:10257000D82EF501C1905F01C826B1F40F5F1F4F3F
:102580000A30110589F78FEF89838A831B820E94A5
:102590000D218160782F9D838C8349815A816B81C5
:1025A0008D810E9434072FC08091960281FD0E9488
:1025B0005915E12CFF24F3948C2D8F21F1F00E940A
:1025C0006D12882399F0EE828F82DF2081E009F47A
:1025D00080E088870E940D218160782F9A87898703
:1025E0004E815F8168858A850E943407F801EC5727
:1025F000FD4F8081F826F08206C0E394FF0CF8E0DE
:10260000EF12DACFBBCF81E0911001C080E02A96B3
:102610000FB6F894DEBF0FBECDBFDF91CF911F91F3
:102620000F91FF90EF90DF90CF90BF90AF909F9071
:102630008F9008950E9494120E94ED180C94020746
:10264000CF93DF930E945714EC01811521E5920787
:1026500008F045C0811530E5930708F094C0883E26
:10266000910528F5803E910508F001C1883A910551
:1026700070F4853A910508F07CC08130910509F429
:1026800075C008F4F1C0049708F0F1C0EDC08F3BAD
:10269000910508F0E9C0C85AD0E0CC0FDD1FC65B39
:1026A000DE4F0990D881C02DCE019464E1C0811520
:1026B00040E2940758F4811551E0950708F0D7C01F
:1026C0008D3E910508F4D0C09065D2C0C11580E45C
:1026D000D80708F4C9C0DF70CE01906AC9C081155F
:1026E00025E59207A8F4811534E5930708F09EC00C
:1026F000811543E5940708F081C0811552E59507DF
:1027000008F064C0D82FCC27CE01816F906AB0C08A
:10271000C11589E5D807A0F4C11528E5D20708F04E
:102720008BC0C11536E5D30708F09EC08C2F0E94E0
:10273000EB148F7190E0D82FCC27CE01906298C017
:10274000C1154AE5D40708F47DC0CE019056811525
:10275000904208F089C08D2F8F710E94EB14DD2705
:10276000D0628F71AE01582BCA0182C081E090E027
:102770007FC0C55AD0E0C858DE4F8881C82FD0E04E
:10278000CE01906475C0F4E096958795FA95E1F7CF
:10279000282F23703C2F337081E090E002C0880F17
:1027A000991F3A95E2F79C68AC01522B9C2F9F70C1
:1027B00096959695892F90E0EC01A5E0CC0FDD1F52
:1027C000AA95E1F7CA018C2B9D2B52C083709927E3
:1027D00021E030E002C0220F331F8A95E2F79C2FE0
:1027E00096959695C92FD0E075E0CC0FDD1F7A95B0
:1027F000E1F7C22BD32BCE019C683AC08370992796
:1028000021E030E002C0220F331F8A95E2F79C2FAF
:1028100096959695C92FD0E065E0CC0FDD1F6A959F
:10282000E1F7C22BD32BCE019A6822C0D82FCC2738
:10283000CE01846F906A1CC0DC2FCC27CE01806F44
:10284000906A16C08C2F8F700E94EB1494E0D6957E
:10285000C7959A95E1F7CF70D0E0DC2FCC27D069EF
:102860009E01282BC90104C080E090E001C0CE0188
:10287000DF91CF9108959B0190E06AE070E00E94A3
:10288000B228830F911DFC0183E0EE0FFF1F8A9594
:10289000E1F7E20FF11DEE0FFF1FE056FF4F8591AC
:1028A000949108950E943B140E9420130895823849
:1028B000910569F1B0F48133910509F46DC048F4D4
:1028C0008932910509F463C08A32910509F469C01F
:1028D00008958533910509F455C089339105B9F000
:1028E0000895833E910569F138F4803E9105B1F079
:1028F000823E910509F10895863E9105A9F1873E32
:102900009105B9F1843E910509F064C023C020917E
:10291000C90220FD4FC021FD4DC008958091C9021C
:1029200080FD44C08091CA0280FF44C08091C902EA
:1029300084FD42C083EE4DC08091C90282FF38C041
:10294000F5CF8091C90282FD33C08091CA0280FD1B
:1029500031C0ECCF8091CA0281FF32C08091C902A0
:1029600084FD2AC087EE35C08091C90283FF26C04E
:10297000F5CF8091C90283FD21C08091CA0281FDFB
:102980001FC0ECCF8091C90285FD1CC01DC0809185
:10299000C90285FD19C016C08091C90286FD16C006
:1029A00017C08091C90286FD13C010C089E311C011
:1029B00082EE0FC080EE0DC080E00BC086EE09C035
:1029C00084EE07C089E205C085E303C08AE201C046
:1029D00081E390E008959091C90292FF0DC0282FE5
:1029E0002871283019F4877F846006C0282F24714D
:1029F000243011F48B7F886093FF0DC0282F28713D
:102A0000283119F4877E846106C0282F247124316F
:102A100011F48B7E88612091CA0220FF0DC0382FEF
:102A20003871383019F4877F816006C0382F3171D2
:102A3000313011F48E7F886021FF0DC0282F28715E
:102A4000283119F4877E816106C0282F2171213138
:102A500011F48E7E886194FD877E089508950E940A
:102A6000A911811102C00E9451120E94B4118093D9
:102A700096020E94BC119093CA028093C9020E94E0
:102A80002E150E94B811682F70E080E090E00E943F
:102A9000B60B6091300270913102809132029091B8
:102AA00033020C94EE0BE82FF0E0EB52FD4F8081E7
:102AB0000895CF92DF92EF92FF920F931F93CF93DF
:102AC000DF9389E991E00E94570585EDE82E82E0C9
:102AD000F82EC0E0D0E094E9C92E91E0D92E0CE8A0
:102AE00011E0DF93CF93DF92CF920E94F00581E94E
:102AF00091E00E945705F70181917F010E94D8065D
:102B00001F928F931F930F930E94F0058AE891E024
:102B10000E94570521968DB79EB708960FB6F89478
:102B20009EBF0FBE8DBFCA30D105D9F6DF91CF91C0
:102B30001F910F91FF90EF90DF90CF90089580EA62
:102B40008A95F1F7089500C008950C949F15089593
:102B50000C94A7150C94A8150C94A7150C94AC15FF
:102B6000F894E82FE295EF70F0E031A1282F2F7054
:102B700081E090E001C0880F2A95EAF7982F9095A0
:102B8000932391A392A1892B82A3789408950F9304
:102B90001F93CF93DF93C3E8D1E089918F3F11F06A
:102BA0000E94B01581E0CD38D807B9F7CBE7D1E066
:102BB00003E811E089918F3F11F00E94B0150C17C6
:102BC0001D07C1F7DF91CF911F910F910895CF920B
:102BD000DF92EF92FF920F931F93CF93DF938C01BD
:102BE000C62FD0E0CE018D579E4F7C01FC01908115
:102BF0009F3F09F447C0D62EF894E92FE295EF7075
:102C0000F0E081A19F7021E030E001C0220F9A9591
:102C1000EAF7822B81A382A12095282322A378940E
:102C20000E94A315EBE7F1E043E851E031E0C12C4D
:102C300021912F3F89F0A22FA295AF70B0E090961E
:102C40008C9190E02F7002C0959587952A95E2F7B8
:102C500080FD02C0832F01C080E0C82A330F4E17C9
:102C60005F0731F7F70180818F3F11F00E94B015A7
:102C700061E0C11001C060E08D2D0E94A515C00F5C
:102C8000D11FC882DF91CF911F910F91FF90EF90DC
:102C9000DF90CF9008950E94C7158AE0E5EDF2E03D
:102CA000DF01982F1D929A95E9F7EBECF2E0DF0136
:102CB0001D928A95E9F78AE00E94AB160C944B06A8
:102CC000FF920F931F93CF93DF93CDB7DEB72A9771
:102CD0000FB6F894DEBF0FBECDBF8E010F5F1F4F42
:102CE0008AE0F80111928A95E9F7F12C6F2DC8015D
:102CF0000E94E715F394FAE0FF12F8CF4AE050E0A3
:102D0000B8018BEC92E00E94FD28FF24F394009719
:102D100009F4F12C892B41F08AE0F801ABECB2E028
:102D200001900D928A95E1F72F2D4AE065ED72E052
:102D30008BEC92E00E94AC160E944D068F2D2A96D5
:102D40000FB6F894DEBF0FBECDBFDF91CF911F91BC
:102D50000F91FF9008950895FF920F931F93CF93C3
:102D6000DF938C01F62ED72FC42F222349F081E068
:102D7000809399020E940D2190939802809397026C
:102D8000809199028823C1F08091970290919802D6
:102D90000E942521059780F0EF2DFD2FD8014C2FA3
:102DA00050E0CD01801B910B841795071CF48D9189
:102DB0008193F7CF10929902DF91CF911F910F91DC
:102DC000FF9008950E94B0230E948C120C94BC23A3
:102DD0000E94C0230E941A130C94DE230E94AB2091
:102DE0000E9497230E947C120E94E2160E94E8161D
:102DF0000E948412FBCF8091A00280FF06C06091E8
:102E0000090170E0660F771F2CC081FF08C0609138
:102E1000090170E0660F771F660F771F22C082FFDF
:102E200009C06091090170E043E0660F771F4A9581
:102E3000E1F717C060919F026623D1F0209108014D
:102E4000621778F78091090190E070E033E0880F15
:102E5000991F3A95E1F70E94B228622F70E00E9414
:102E6000CF286038710540F46115710519F406C06A
:102E700068E070E0862F08958FE7089581E0089557
:102E80008091A00280FF08C06091050170E07595F7
:102E900067957595679523C081FF06C06091050110
:102EA00070E0759567951BC082FF04C060910501B5
:102EB00070E012C060919E026623A9F02091040187
:102EC0006217A0F78091050170E090E00E94B2289F
:102ED000622F70E00E94CF286038710540F46115C0
:102EE000710519F406C061E070E0862F08958FE740
:102EF000089581E008958D3E21F40E94FB1681958E
:102F000004C08E3E29F40E94FB168093A40208950B
:102F10008F3E21F40E94FB16819504C0803F29F466
:102F20000E94FB168093A3020895893F19F40E9422
:102F3000401705C08A3F31F40E9440178195809365
:102F4000A50208958B3F21F40E944017819504C08B
:102F50008C3F29F40E9440178093A60208959FE0B9
:102F6000980F983078F421E030E0A90102C0440FB6
:102F7000551F9A95E2F7CA019091A202892B80937E
:102F8000A20208958D3F21F48091A00281600BC0C0
:102F90008E3F21F48091A002826005C08F3F29F40A
:102FA0008091A00284608093A00208958D3E39F440
:102FB0009091A40297FF35C01092A40259C08E3E92
:102FC00029F49091A4021916BCF32BC09091A3028E
:102FD0008F3E29F497FF25C01092A30249C0803F7D
:102FE00019F41916CCF31DC09091A502893F29F45C
:102FF0001916BCF41092A5023BC08A3F19F497FF42
:1030000010C0F8CF8B3F39F49091A60297FF09C00A
:103010001092A6022DC08C3F21F49091A6021916A1
:10302000BCF39FE0980F983080F421E030E0A901D4
:1030300002C0440F551F9A95E2F7CA0180959091FE
:10304000A20289238093A20213C08D3F21F48091B4
:10305000A0028E7F0BC08E3F21F48091A0028D7F55
:1030600005C08F3F29F48091A0028B7F8093A0023E
:103070008091A302811106C08091A402811102C037
:1030800010929F028091A502811106C08091A60234
:10309000811102C010929E0208958091960283FFD2
:1030A0007EC08FEC91E00E9457058091A2021F9292
:1030B0008F938AEC91E09F938F930E94F00588ECA8
:1030C00091E00E9457058091A302282F082E000C42
:1030D000330B3F938F9385EC91E09F938F930E94E6
:1030E000F00583EC91E00E9457058091A402282FFF
:1030F000082E000C330B3F938F9380EC91E09F934D
:103100008F930E94F0058EEB91E00E94570580910D
:10311000A502282F082E000C330B3F938F938BEBC7
:1031200091E09F938F930E94F00589EB91E00E94BC
:1031300057058091A602282F082E000C330B3F93D1
:103140008F9386EB91E09F938F930E94F00583EB22
:1031500091E00E94570580919F021F928F9380EB10
:1031600091E09F938F930E94F0058EEA91E00E9478
:1031700057058091A0021F928F938BEA91E09F9355
:103180008F930E94F00588EA91E00E9457058DB761
:103190009EB74C960FB6F8949EBF0FBE8DBF0E948F
:1031A0000D212091A302211104C02091A402222309
:1031B00021F090939D0280939C022091A502211101
:1031C00004C02091A602222321F090939B028093B9
:1031D0009A0281EA92E00C94EB1FEF92FF920F9318
:1031E0001F93CF93DF9300D000D000D0CDB7DEB7D0
:1031F00086E0E1EAF2E0DE01119601900D928A95F7
:10320000E1F7E090A302F090A4020091A5021091D2
:10321000A6021092A3021092A4021092A50210928C
:10322000A602E11003C0FF2009F464C080919C0253
:1032300090919D020E942521FC0120919F02222352
:1032400039F080910A0190E08E179F0760F052C01C
:1032500080910B0190E06AE070E00E94B2288E1726
:103260009F0718F047C02F3F19F02F5F20939F0250
:10327000EE2061F00E94FB16682F1E1414F08FEFF1
:1032800001C081E00E94A9288093A302FF2061F081
:103290000E94FB16682F1F1414F08FEF01C081E00D
:1032A0000E94A9288093A4028091A302882311F18F
:1032B0002091A4022223F1F0082E000C990B65EB5B
:1032C00070E00E94B228992319F09093A30203C0E2
:1032D00081E08093A302822F220F990B65EB70E0AF
:1032E0000E94B228992319F09093A40203C081E0B0
:1032F0008093A402011103C0112309F464C08091DA
:103300009A0290919B020E942521FC0120919E022D
:10331000222339F08091060190E08E179F0760F01C
:1033200052C08091070190E06AE070E00E94B228EC
:103330008E179F0718F047C02F3F19F02F5F20937B
:103340009E02002361F00E944017682F101614F0AF
:103350008FEF01C081E00E94A9288093A50211236C
:1033600061F00E944017682F111614F08FEF01C012
:1033700081E00E94A9288093A6028091A50288235B
:1033800011F12091A6022223F1F0082E000C990BD6
:1033900065EB70E00E94B228992319F09093A50282
:1033A00003C081E08093A502822F220F990B65EB69
:1033B00070E00E94B228992319F09093A60203C0EE
:1033C00081E08093A6028091A30281110BC08091BD
:1033D000A402811107C08091A502811103C08091D0
:1033E000A60281110E944D18EB82FC820D831E8380
:1033F00086E0FE013196A1EAB2E001900D928A9535
:10340000E1F726960FB6F894DEBF0FBECDBFDF9171
:10341000CF911F910F91FF90EF900895E1EAF2E0B4
:1034200086E0DF011D928A95E9F710929F021092C3
:103430009E021092A0020895CF93DF93EC01FB014E
:103440008281882309F43CC1C430FDE5DF0760F4C4
:10345000CB3F9CE5D90788F49E0122503C4524319E
:10346000310508F02EC109C0C236EDE5DE0729F0AE
:10347000C63AFDE5DF0709F024C10E94BC11909314
:10348000CA028093C902C1318CE5D80709F4C6C0CD
:1034900008F042C0C930ECE5DE0709F49BC000F536
:1034A000C5308CE5D80709F485C078F4C330ECE565
:1034B000DE0709F478C008F07AC0C230DC4509F0B4
:1034C000F5C08091C9028160EFC0C7309CE5D90783
:1034D00009F478C008F07AC08091C9028061E4C024
:1034E000CD30FCE5DF0709F487C058F4CB309CE50C
:1034F000D90709F479C008F07BC08091C9028860BF
:103500006FC0CF30FCE5DF0709F480C008F082C04F
:103510008091C902877FC8C0CE3F9CE5D90709F4D6
:1035200071C000F5C531FCE5DF0709F485C068F41A
:10353000C3319CE5D90709F475C008F095C00E9415
:103540005E0B8091C9028F77AFC0CC3FFCE5DF07EF
:10355000A9F108F054C0CB3FDC4509F0A7C0809129
:10356000CA0240C0C230EDE5DE0709F489C058F454
:10357000C1158DE5D80709F45AC008F069C08091DB
:10358000CA0282602FC0C236EDE5DE0709F47CC0B6
:10359000C63AFDE5DF0709F481C0C330DD4509F017
:1035A00085C080E06EC08091C90282607DC080913C
:1035B000C90216C08091C902886076C08091CA0293
:1035C00082604FC08091C90280626EC08091C90242
:1035D00080646AC00E945E0B8091C902806864C0EA
:1035E000846062C081603DC08091C9028E7F5CC0F2
:1035F0008091C9028D7F58C08091C90216C0809108
:10360000CA0218C08091CA028D7F2BC08091C90266
:103610008F7E4AC08091C9028F7D46C08091C902C9
:103620008F7B42C08091C902877F8B7F3DC0809194
:10363000CA028D7F8E7F15C08091C90282FB22272E
:1036400020F991E0922790FB82F990FB83F92CC03E
:103650008091CA02982F909591708E7F892B90FB54
:1036600081F98093CA0222C00E945E0B8091C90238
:1036700087FB222720F991E0922790FB87F914C05D
:1036800081E00E94531212C08091C90284FB22275C
:1036900020F991E0922790FB84F906C08091C9023D
:1036A000982F909590FB80F98093C9028091C90270
:1036B0009091CA020E94CD110E945E0B80E001C071
:1036C00081E0DF91CF910895809104011F928F9343
:1036D000809105011F928F93809108011F928F9313
:1036E000809109011F928F9380910A011F928F93FD
:1036F00080910B011F928F9382EF91E09F938F93A4
:103700000E94F0058DB79EB70E960FB6F8949EBF37
:103710000FBE8DBF0895883220F58E3108F068C045
:103720008B3091F1C0F4873009F0BEC081E0809306
:103730000B0184E180930A018AE0809309018EE104
:103740008093080188E08093050188E2809304015A
:1037500084E593E0C6C0833109F443C0843169F144
:10376000A3C08F3409F49EC028F4893231F1883324
:1037700059F09AC0813531F008F4D4C0823509F48B
:10378000A7C092C08FEFA5C086E793E00E945705BF
:103790000E94641B1F9281E08F931F9288E08F9399
:1037A0008FE692E09F938F930E94F0050F900F9009
:1037B0000F900F900F900F9096C083E793E00E94B8
:1037C00057058091AB02882309F4AAC01092AB027E
:1037D0001092AA021092A9021092A8021092A702B7
:1037E000B1C085E693E00E9457050E94641B7BC030
:1037F0008D518093AB02833031F170F48130D1F080
:10380000823009F03FC08AE091E09093AA02809351
:10381000A9028AE991E01FC0853059F108F186308C
:1038200089F584E091E09093AA028093A90285ED46
:1038300091E011C08BE091E09093AA028093A902DD
:1038400081E991E008C089E091E09093AA02809319
:10385000A90286EA91E09093A8028093A70218C07B
:1038600088E091E09093AA028093A90283EB91E013
:10387000F2CF85E091E09093AA028093A90282ECB6
:1038800091E0E9CF1092AB0282E693E00E945705E7
:103890008091AB02882309F455C01F928F938EE567
:1038A00093E00DC08AE015C081E593E01AC097FF50
:1038B00047C0108280811F928F938BE493E09F9387
:1038C0008F930E94F0050F900F900F900F900BC0F8
:1038D00081E0E091A902F091AA02309729F588E4ED
:1038E00093E00E9457052091AB02222359F1809169
:1038F000A7029091A802009711F48DE891E09F93A0
:103900008F931F922F938FE393E09F938F930E9447
:10391000F0050F900F900F900F900F900F9016C022
:1039200080E0089586EFD5CF2081082E000C990BFA
:10393000820F911D8F3F910509F00CF4B8CF8FEFE6
:103940008083B8CF8BE393E00E94570581E0089510
:10395000CF93C82F1F928F938CE893E09F938F9300
:103960000E94F00581E090E0A0E0B0E0BC01CD0154
:1039700004C0660F771F881F991FCA95D2F70E944F
:10398000B60B0F900F900F900F90CF910C945E0B91
:10399000EF92FF920F931F93CF93DF938B3109F434
:1039A000EDC008F08EC08B3009F4B1C008F078C0CB
:1039B000863009F4AFC020F4853009F4BDC04EC193
:1039C000873009F4C0C0883009F048C10E94B8119E
:1039D0001F928F9388EB97E09F938F930E94F0053F
:1039E0000E94B41183FB992790F91F929F9382FB49
:1039F000992790F91F929F9381FB992790F91F9225
:103A00009F93982F91701F929F931F928F938FE691
:103A100097E09F938F930E94F0050E94BC1187FB53
:103A2000222720F91F922F9386FB222720F91F922D
:103A30002F9385FB222720F91F922F9384FB2227A7
:103A400020F91F922F9383FB222720F91F922F9397
:103A500082FB222720F91F922F9391FB222720F926
:103A60001F922F93292F21701F922F9381FB2227C2
:103A700020F91F922F93282F21701F922F939F932D
:103A80008F938AE896E09F938F930E94F0058DB7FD
:103A90009EB788960FB6F8949EBF0FBE8DBF35C0F7
:103AA000803109F495C020F48E3009F47BC0D6C073
:103AB000863109F4A8C0893109F0D0C08CEF93E0B9
:103AC00084C08A32E1F060F4873209F4C3C028F47C
:103AD0008E3108F4C3C08D51BEC0893269F1BEC0B9
:103AE000833448F48A3308F0B3C0853309F4B2C094
:103AF000883369F0B3C0833409F4ACC0AFC083E647
:103B000098E00E9457050E945112C1E0ACC087EEB8
:103B100094E05BC080919602817F8E7F80939602B5
:103B200080EC94E00E9457058FE598E00E945705CD
:103B300081E08093AC02E9CF83E498E00E945705CE
:103B40000E945006E2CF80919602C82FC095C170A6
:103B5000C0FB80F980939602CC2329F087E398E09C
:103B60000E94570580C08AE298E00E945705809124
:103B70009602897F877F80939602C7CF90919602A5
:103B800091FBCC27C0F981E0C827892FC0FB81F9C0
:103B900080939602CC2319F08DE198E029C08FE044
:103BA00098E013C09091960292FBCC27C0F981E077
:103BB000C827892FC0FB82F980939602CC2319F085
:103BC00080E098E015C080EF97E00E9457059DCFF8
:103BD0009091960293FBCC27C0F981E0C827892FEA
:103BE000C0FB83F980939602CC2351F084EE97E0DA
:103BF0000E9457058091960281608093960233C09F
:103C000087ED97E0E2CF0E941921162F072FF82E9B
:103C1000E92ED091C802C09118010E94961FEF9220
:103C2000FF920F931F931F92DF931F92CF931F92C8
:103C30008F9381E993E09F938F930E94F0058DB756
:103C40009EB70C960FB6F8949EBF0FBE8DBF5DCF8A
:103C5000895301C080E00E94A81C57CF85ED97E0F2
:103C60000E945705C0E08C2FDF91CF911F910F91DB
:103C7000FF90EF90089580E008950C943B1ECF9341
:103C8000C82F8091AC02813071F040F0823009F091
:103C900045C08C2F0E948B1B81E046C00E94B21051
:103CA0008232F1F504C00E94B210823261F48C2F8E
:103CB0000E943D1E811104C08C2F0E94C81C2CC084
:103CC00081E090E029C08C2F0E943B1E811123C00F
:103CD000C431C9F058F4CB3069F0C031B9F482E096
:103CE0008093AC0288E30E948B1B15C0C93259F047
:103CF000C83361F480EC94E00E94570588E893E0B3
:103D00000E94570508C01092AC020CC086E893E0F0
:103D10000E94570507C081E0817006C01092AC0276
:103D200080E002C080E0F8CFCF910895CF93DF9379
:103D300086319C4541F5EB010E94B210982F8A8193
:103D40002091020130910301882379F09A7A81E071
:103D500009F480E08093AD02911102C069E201C0D4
:103D600065E3C9010E9467200AC08091AD028111FC
:103D700002C069E201C065E3C9010E9469200E9496
:103D8000F41080E001C081E0DF91CF9108950F939E
:103D90001F93CF93DF93C42FD22FFC0182818823FE
:103DA000C9F04093B0020E940D219093AF0280931E
:103DB000AE0280E28C0F883008F057C0C77081E0F7
:103DC00001C0880FCA95EAF7DF91CF911F910F913B
:103DD0000C94BB088091B002481330C08091AE02B1
:103DE0009091AF020E942521883C910538F510E2A0
:103DF0001D0FCD17B9F080E28C0F883040F4C770EA
:103E000081E001C0880FCA95EAF70E94C208183005
:103E100028F581E09D2F977001C0880F9A95EAF7E9
:103E20000E94BB08802F0E94B2081830F0F4D770AF
:103E300081E001C0880FDA95EAF70AC080E28C0FB2
:103E4000883098F4C77081E001C0880FCA95EAF7FE
:103E5000DF91CF911F910F910C94C208802FDF91B9
:103E6000CF911F910F910C94B208DF91CF911F91C8
:103E70000F9108950F939C01CB01243F4CE534072B
:103E800031F188F4293DFCE53F07D9F02A3D4CE5A6
:103E9000340779F1283D3C45A9F506E221EE41EED3
:103EA00068ED7CE52BC0263FFCE53F07E1F0A8F07C
:103EB000273F3C4539F507E225EE46EE67EF7CE506
:103EC0001DC007E225EE45EE69ED7CE517C006E270
:103ED00021EE40EE64EF7CE511C007E225EE44EEF2
:103EE00065EF7CE50BC006E221EE42EE66EF7CE575
:103EF00005C008E221E045EE6AED7CE50E94C71EA0
:103F000080E008C0FC018281882319F01092B00281
:103F100001C081E00F9108959093FB018093FA0115
:103F200008959093B6028093B5020895E091B5028A
:103F3000F091B602309721F00190F081E02D0994C4
:103F400080E00895EF92FF920F931F93CF93DF933A
:103F5000E091B502F091B6023097B1F18C01028088
:103F6000F381E02D09958091960282FF2DC080FF9C
:103F700004C08CE798E00E945705E80118E086E746
:103F8000E82E88E0F82E8091960280FF0BC0888191
:103F90001F928F93FF92EF920E94F0050F900F9067
:103FA0000F900F90115021961111EDCF8091960234
:103FB00080FF0AC084E798E0DF91CF911F910F91B5
:103FC000FF90EF900C945705DF91CF911F910F91C7
:103FD000FF90EF900895E091B502F091B60230970E
:103FE00039F022E0DC012C930480F581E02D099466
:103FF00008952091B3023091B4022817390771F067
:104000009093B4028093B302E091B502F091B602AE
:10401000309721F00680F781E02D099408952091D2
:10402000B1023091B2022817390771F09093B202B1
:104030008093B102E091B502F091B602309721F081
:104040000084F185E02D09940895FC01329697E0F3
:1040500080E0915029F021912223D9F38F5FF9CF8D
:104060000895662349F0FC01329608962191621763
:1040700029F0E817F907D1F780E0089581E0089565
:104080009C01FC0132969FEF80E04191461789F038
:104090009F3F19F4411101C0982F8F5F8630A9F717
:1040A0009F3F39F0F901E90FF11D97FDFA95628301
:1040B000089508959C012A5F3F4FFC0142814613F9
:1040C00001C01282019682179307B9F708950C94E4
:1040D00040200C945A20029626E0FC0111922A9569
:1040E000E9F7089508950C94722083E08093B70255
:1040F0000C947320811102C081E001C082E08093A2
:10410000B7020C9473200C947A2081E08093B7025C
:104110000C9473200C94852008950C948C200C949E
:104120008D200C948C200C948C200C948C20CF939C
:104130000E9493200E9460160E949120C0E08C2F64
:104140000E945315811104C0CF5FCA30C1F701C06E
:1041500081E0CF91089508951F920F920FB60F92AC
:1041600011248F939F93AF93BF938091B8028111D5
:1041700013C08091DF029091E002A091E102B09122
:10418000E2024196A11DB11D8093DF029093E002EF
:10419000A093E102B093E202BF91AF919F918F9102
:1041A0000F900FBE0F901F9018958091E7028430FA
:1041B00031F10E94D0061092B80220E488E190E02C
:1041C0000FB6F894A895809360000FBE209360000E
:1041D00083B7817F846083BF83B7816083BF789416
:1041E000889583B78E7F83BF0FB6F894A89580918A
:1041F0006000886180936000109260000FBE089597
:104200000E945E0B0C94D40682E084BD93E095BDC1
:104210009AEF97BD80936E0008952FB7F894809120
:10422000DF029091E002A091E102B091E2022FBF83
:1042300008952FB7F8946091DF027091E0028091A9
:10424000E1029091E2022FBF08959C014FB7F894CC
:104250008091DF029091E002A091E102B091E20230
:104260004FBF821B930B089578941F920F920FB645
:104270000F9211248F939F93AF93BF938091DF028E
:104280009091E002A091E102B091E2020196A11D9D
:10429000B11D8093DF029093E002A093E102B093FE
:1042A000E202BF91AF919F918F910F900FBE0F903F
:1042B0001F90189581E08093E00080E28093D80001
:1042C0001092C9008FE19EE40197F1F700C0000051
:1042D00087E090EBDC018093F0029093F102A093D1
:1042E000F202B093F3029CE088E10FB6F894A8952F
:1042F000809360000FBE90936000FFCF8091C70253
:104300000895089522E02093E9002FEF3091E8000E
:10431000215035FD06C035ED3A95F1F70000211129
:10432000F5CF2091E80025FF0BC040E050E066E0AB
:1043300070E00E944D248091E8008E778093E80021
:104340000895CF93DF9321E02093E9002FEF309180
:10435000E800215035FD06C035ED3A95F1F7000033
:104360002111F5CF2091E80025FF14C0EC0140E0B9
:1043700050E068E070E00E944D248091E8008E7764
:104380008093E80088E0FE01AFEBB2E001900D926F
:104390008A95E1F7DF91CF9108958093BB027093E6
:1043A000BD026093BC028091E702843001F582E097
:1043B0008093E9008FEF9091E800815095FD06C051
:1043C00095ED9A95F1F700008111F5CF8091E80005
:1043D00085FF0DC040E050E063E070E08BEB92E0C1
:1043E0000E944D248091E8008E778093E800089524
:1043F000BC0184E00C94CD21BC0183E00C94CD2160
:104400008AE998E00E9457050C948A2086E998E092
:104410000E9457056091E30281E0611101C080E0D4
:104420000C94752082E998E00E9457059091E7026C
:1044300081E0943009F080E06091E3020C947A20EE
:104440002091BA022F5F822F62E30E94C328992332
:1044500019F02093BA0208951092BA028091BE0218
:10446000882371F18091E702843041F58091E90061
:104470008F702091EC00922F917020FD90E8892B95
:1044800093E09093E9009091EB0090FF14C090911D
:10449000EE0097FF10C09091E80095FF03C01092C6
:1044A000F100F9CF9091E80090FF05C09091E800ED
:1044B0009E779093E8008F708093E9001092BE027F
:1044C000089542E061EC81E00E94512542E261ECF6
:1044D00082E00E94512542E261EC83E00E94512576
:1044E0009091E70281E0943009F080E06091E3026E
:1044F0000C9483208091E902833009F45DC030F48C
:10450000813071F0823009F496C008958A3009F440
:1045100082C08B3009F468C0893009F0A4C020C083
:104520008091E802813A09F09EC08091E800877F7F
:104530008093E8008091EC029091ED02892B21F4A8
:1045400068E08FEB92E003C060E080E090E070E014
:104550000E9498248091E8008B778093E80008956A
:104560008091E802813209F07EC08091EC02909146
:10457000ED02029708F077C08091E800877F809372
:10458000E8008091E80082FD05C08091E70281117A
:10459000F8CF69C08091F200823031F48091F1004F
:1045A000813011F0863021F48091F1008093C702B0
:1045B0008091E8008B7753C08091E802813A09F03E
:1045C00052C08091EC029091ED02892B09F04BC012
:1045D0008091E800877F8093E8008091E80080FF69
:1045E000FCCF8091180136C08091E8028132D9F564
:1045F0008091EC029091ED02892BA9F58091E80061
:10460000877F8093E8000E9486258091EA0280934C
:1046100018010C945E0B8091E802813221F58091A3
:10462000E800877F8093E8000E9486258091EB0256
:104630008093C80208958091E802813AA1F48091A4
:10464000E800877F8093E8008091E80080FFFCCF3E
:104650008091C8028093F1008091E8008E7780936A
:10466000E8000C94862508959FB7F8941092BE0236
:104670009FBF9091E702943009F057C09091E900F4
:104680009F703091EC00232F217030FD20E8922B99
:1046900023E02093E9002091EB0020FF43C020910C
:1046A000EE0027FF3FC02091B902222321F0209184
:1046B000E80025FF37C01092B90226E03091E800EB
:1046C00035FD15C03091E702343061F53091EB00D3
:1046D00035FD28C0215021F481E08093B90222C029
:1046E000EFE9FFE03197F1F700C00000E7CF8093DA
:1046F000F1008091E80085FD0AC08091E80080FF0C
:10470000FCCF8091E8008E778093E80006C08FB7D9
:10471000F89421E02093BE028FBF9F709093E90030
:1047200080E008959F709093E9008FEF089584B71B
:10473000877F84BF0FB6F894A89580916000886148
:1047400080936000109260000FBE90E080E80FB68A
:10475000F89480936100909361000FBE0C948520C3
:104760000E94D8250E942B26E2EEF0E08081846032
:10477000808378940C948E288CE091E00C94911FA7
:104780008091E7028530C9F48EE898E00E945705D1
:104790008091E702853079F40E94D5208091E5026E
:1047A0008823B1F30E949720882391F30E94372435
:1047B0000E945E0BEDCF0C940021089508950C9497
:1047C000E123292F332723303105C9F060F421304C
:1047D000310581F02230310509F041C08BE590E0D0
:1047E00028ED38E040C021323105E1F022323105B8
:1047F00031F135C082E190E023E339E034C09927FC
:104800008130910549F028F0029749F5EEE9F8E08A
:1048100005C0E4EDF8E002C0EAEAF8E0849190E037
:104820009F0121C063307105D0F4660F771FFB0133
:10483000ED50FE4F2081318189E090E014C063305B
:10484000710568F4FB01EE0FFF1FE351FE4F20815D
:104850003181FB01E651FE4F808190E004C080E091
:1048600090E020E030E0FA0131832083089584E075
:1048700089BD86E089BD09B400FEFDCF8091D800D6
:104880008F7D8093D8008091E00082608093E0006B
:104890008091E00081FDFCCF0895CF92DF92EF92EE
:1048A000FF920F931F93CF93DF93EC018B017A015B
:1048B0000E94A525811133C0E114F10439F0F701FC
:1048C00080819181081B190BC80FD91FC12CD12CD5
:1048D0000115110519F18091E80085FD16C0809140
:1048E000E8008E778093E800E114F10449F0F701C5
:1048F00080819181C80ED91ED182C08285E00FC00F
:104900000E94A525882321F30AC089918093F10094
:1049100001501109FFEFCF1ADF0ADACF80E0DF91F3
:10492000CF911F910F91FF90EF90DF90CF9008955E
:104930002091EE023091EF022617370748F06115FB
:10494000710539F42091E8002E772093E80001C02A
:10495000B901FC0120E06115710561F18091E70268
:104960008823D9F18530D9F18091E80083FD39C0E1
:104970008091E80082FD2BC08091E80080FFEBCFA2
:104980008091F20090E06115710551F08830910539
:1049900038F421912093F100615071090196F3CF11
:1049A00021E0089709F020E08091E8008E7780935D
:1049B000E800D1CF2111D2CF0AC08091E70288232D
:1049C00061F0853061F08091E80083FD0AC080913C
:1049D000E80082FFF2CF80E0089582E0089583E04E
:1049E000089581E008952091EE023091EF0226179C
:1049F000370748F06115710539F42091E8002E77EA
:104A00002093E80001C0B901FC0120E061157105A7
:104A100079F18091E702882309F43DC0853009F4DB
:104A20003CC08091E80083FD3AC08091E80082FD9F
:104A30002CC08091E80080FFE9CF8091F20090E0E7
:104A40006115710559F08830910540F42491209347
:104A5000F1003196615071090196F2CF21E008977B
:104A600009F020E08091E8008E778093E800CECFB7
:104A70002111CFCF0AC08091E702882361F08530F1
:104A800061F08091E80083FD0AC08091E80082FF18
:104A9000F2CF80E0089582E0089583E0089581E0F8
:104AA0000895982F953068F59093E900981739F09C
:104AB0007091EC002091ED005091F00003C0242F84
:104AC000762F50E021FD02C09F5FECCF3091EB00CC
:104AD0003E7F3093EB003091ED003D7F3093ED0051
:104AE0003091EB0031603093EB007093EC00209339
:104AF000ED005093F0002091EE0027FDE5CF80E01F
:104B000008958F708093E90081E008958091E80214
:104B100087FF11C08091E80082FD05C08091E70207
:104B20008111F8CF11C08091E8008B770BC0809184
:104B3000E702882349F08091E80080FFF8CF809158
:104B4000E8008E778093E80008952091E40030918A
:104B5000E50095E64091EC00842F817040FF23C072
:104B60008091E80080FD1DC08091E702882399F0C4
:104B7000853099F08091EB0085FD11C04091E400F3
:104B80005091E5002417350729F3915011F09A014F
:104B9000E1CF84E0089582E0089583E0089581E004
:104BA000089580E008954091E80042FFDDCF089528
:104BB0000E9435260E943826E0EEF0E08081816078
:104BC0008083E8EDF0E080818F77808319BCE3E695
:104BD000F0E08081816080831092E60208950E9457
:104BE00035260E9438268091D8008F778093D80090
:104BF0008091D80080688093D8008091D8008F7D04
:104C00008093D80084E089BD86E089BD09B400FEA8
:104C1000FDCF1092E7021092E3021092E50210928B
:104C2000E40242E060E080E00E9451258091E100D2
:104C30008E7F8093E1008091E20081608093E200AA
:104C40008091E20088608093E2008091E0008E7F96
:104C50008093E0000895E3E6F0E080818E7F80831A
:104C600081E08093E6020C94EF251092E200089513
:104C70001092E10008951F920F920FB60F92112427
:104C80002F933F934F935F936F937F938F939F9354
:104C9000AF93BF93EF93FF938091E10082FF0BC02E
:104CA0008091E20082FF07C08091E1008B7F8093BA
:104CB000E1000E9420228091E10080FF19C08091D4
:104CC000E20080FF15C08091E2008E7F8093E200B9
:104CD0008091E20080618093E2008091D800806240
:104CE0008093D80019BC85E08093E7020E940622D9
:104CF0008091E10084FF30C08091E20084FF2CC0ED
:104D000084E089BD86E089BD09B400FEFDCF8091B5
:104D1000D8008F7D8093D8008091E1008F7E8093B2
:104D2000E1008091E2008F7E8093E2008091E200BA
:104D300081608093E2008091E302882311F084E097
:104D400007C08091E30087FD02C081E001C083E0DD
:104D50008093E7020E9412228091E10083FF29C024
:104D60008091E20083FF25C08091E100877F8093DE
:104D7000E10082E08093E7021092E3028091E1007B
:104D80008E7F8093E1008091E2008E7F8093E2002D
:104D90008091E20080618093E20042E060E080E088
:104DA0000E9451258091F00088608093F0000E945D
:104DB0000022FF91EF91BF91AF919F918F917F91D1
:104DC0006F915F914F913F912F910F900FBE0F9078
:104DD0001F9018951F920F920FB60F9211242F93C8
:104DE0003F934F935F936F937F938F939F93AF9373
:104DF000BF93CF93DF93EF93FF93C091E900CF7000
:104E00008091EC00D82FD17080FDD0E81092E9009D
:104E10008091F000877F8093F00078940E942E2785
:104E20001092E9008091F00088608093F000CD2B13
:104E3000CF70C093E900FF91EF91DF91CF91BF91C7
:104E4000AF919F918F917F916F915F914F913F9122
:104E50002F910F900FBE0F901F9018951F93CF9317
:104E6000DF93CDB7DEB7AA970FB6F894DEBF0FBEBB
:104E7000CDBFE8EEF2E08091F100819322E0E03FC7
:104E8000F207C9F70E947A228091E80083FF2EC1C1
:104E90008091E8029091E902492F50E04A30510593
:104EA00008F024C1FA01EA5BFF4F0C94E328803834
:104EB00021F0823809F01AC108C08091E402909173
:104EC000E502992389F082600FC08091EC028F7017
:104ED000853008F00BC18093E9008091EB0085FBE1
:104EE000882780F91092E9009091E800977F9093CD
:104EF000E8008093F1001092F100D1C0282F2D7F9F
:104F000009F0F4C0882319F0823061F0EFC080917D
:104F1000EA02813009F0EAC0933009F080E0809322
:104F2000E5022EC08091EA0281112AC08091EC0234
:104F30008F702FEF280F243008F0D8C08093E9003D
:104F40002091EB0020FF1CC0933021F48091EB00F6
:104F5000806214C09091EB0090619093EB0021E08F
:104F600030E0A90102C0440F551F8A95E2F7409333
:104F7000EA001092EA008091EB0088608093EB00D9
:104F80001092E9008091E800877F8093E8000E94FA
:104F90008625ACC08111AAC01091EA021F778091CA
:104FA000E3008078812B8093E3008091E800877F85
:104FB0008093E8000E9486258091E80080FFFCCF66
:104FC0008091E30080688093E300111102C082E0C9
:104FD00001C083E08093E70289C08058823008F0E6
:104FE00085C08091EA029091EB028C3D53E09507D9
:104FF00079F583E08A838AE289834FB7F894DE01EA
:10500000139620E03EE051E2E32FF0E0509357008A
:10501000E49120FF03C0E295EF703F5FEF708E2FA9
:1050200090E0EA3010F0C79601C0C0968D939D9332
:105030002F5F243149F74FBF8091E800877F80932D
:10504000E8006AE270E0CE0101960E94982416C042
:105050006091EC027091ED02AE014F5F5F4F0E94D4
:10506000DF23BC01892B09F441C09091E800977FB0
:105070009093E80089819A810E94F3248091E8004E
:105080008B778093E80032C0803881F58091E8000A
:10509000877F8093E8008091E3028093F100809104
:1050A000E8008E7772CF811121C08091EA02909141
:1050B000EB0299270297D4F48091E800877F8093D0
:1050C000E8008091EA028093E3020E9486258091A5
:1050D000E302811106C08091E30087FD02C081E0F8
:1050E00001C084E08093E7020E9461228091E80081
:1050F00083FF0AC08091E800877F8093E800809159
:10510000EB0080628093EB00AA960FB6F894DEBFA6
:105110000FBECDBFDF91CF911F910895CF938091A6
:10512000E7028823A1F0C091E900CF709091EC00D4
:10513000892F817090FD80E8C82B1092E900809142
:10514000E80083FD0E942E27CF70C093E900CF9125
:105150000895002480FD060E660F11F08695D1F7A4
:10516000802D08950024552704C0080E591F880F6C
:10517000991F009729F076956795B8F37105B9F7EF
:10518000802D952F0895991B79E004C0991F9617DB
:1051900008F0961B881F7A95C9F78095089597FBAC
:1051A000072E16F4009407D077FD09D00E94E92855
:1051B00007FC05D03EF4909581959F4F089570951A
:1051C00061957F4F0895EE0FFF1F0590F491E02D3C
:1051D0000994AA1BBB1B51E107C0AA1FBB1FA6173E
:1051E000B70710F0A61BB70B881F991F5A95A9F790
:1051F00080959095BC01CD010895FB01DC0104C0B0
:105200008D910190801921F441505040C8F7881BBE
:10521000990B0895F999FECF92BD81BDF89A99270F
:1052200080B50895A8E1B0E042E050E00C943E293A
:10523000262FF999FECF92BD81BDF89A019700B44F
:10524000021639F01FBA20BD0FB6F894FA9AF99AEF
:105250000FBE08950396272F0E9419290E9418292E
:10526000252F0E941929242F0C9419290196272FE4
:105270000E9419290C941829DC01CB01FC01F99931
:10528000FECF06C0F2BDE1BDF89A319600B40D9292
:0C52900041505040B8F70895F894FFCF4B
:10529C00C8007A02280850011E0A14017E21A1219F
:1052AC008221FC21F821812101E200E900EA00B50C
:1052BC0000B600B700CD008301CC008A01920194A6
:1052CC00012102230224022502260227022A02B30C
:1052DC0000B4006F007000818283E200E900EA00F4
:1052EC00B500B600B700CD008301CC008A01920155
:1052FC0094012102230224022502260227022A02FB
:10530C00B300B4006F0070008182839392353667CE
:10531C00666564629091949596303132333F3F3F8D
:10532C00006D6B5F64656C6179006D6B5F696E74A9
:10533C00657276616C006D6B5F6D61785F73706523
:10534C006564006D6B5F74696D655F746F5F6D6133
:10535C0078006D6B5F776865656C5F6D61785F7306
:10536C0070656564006D6B5F776865656C5F74690B
:10537C006D655F746F5F6D617800407B22E2096739
:0A538C00094509EA0803091C09009D
:00000001FF
